:020000040000FA
:08000800052883120313850192
:1000100086010F308700880189018316FF30850033
:1000200086010030870088018901863081008312B3
:100030001F3087006A25F028820747345234413444
:10004000503448344934433420344C3443344434F9
:100050002034443445344D344F34453450344534E1
:100060002034533448344F345734533420345934C3
:100070004F345534203448344F34573421345434B9
:1000800048344934533420344934533420345034C0
:1000900041344734453420343234513455344134BA
:1000A00043344B348207803483348634833483343E
:1000B000813482348334863483348B348734893476
:1000C000003481348434003487348C348D34883463
:1000D0000034853488348A348E3482078034C034C6
:1000E000A034903488348434823481348034803431
:1000F00080348034803480348034803480344034A0
:100100002034103408340434023401340034003410
:1001100000340034003400340034FF34013402343D
:100120000434083410342034403480348134823430
:10013000843488349034A034C034803400340034A3
:100140007A344A344A344A344A34CB344A344A340E
:100150004A344A344A347A3400340034083404349B
:1001600002340134023404340834103402340234CA
:1001700002340234023404340834103408340434B1
:1001800002340234023402340234003400340034C5
:1001900092349A349634923400340034003400346B
:1001A00032344A344A3431340034003400340034B8
:1001B0005F344434443484340034003400346534CF
:1001C00095349534623400340034003407398207A2
:1001D0008034403420341034083404340234013480
:1001E0002230AD007C250C21632556216625C521D2
:1001F0006325E5216325EE21662513226625292244
:100200006325682266251623632526236325492353
:100210006625C4236625F028943011257830A10086
:100220009F24A801053047250130A100A001C62464
:10023000A801013044250930A100C624A8010130DD
:1002400041250A30A100C624A80103303E25033011
:10025000A100C624A80103303B250130A100C6241B
:10026000A801033038250130A100C624A8010330BD
:1002700035250130A100C624A80100304A251030E0
:10028000A100A001AF24A801063038250A30A10042
:10029000AF24A801063035250830A100AF24A801FD
:1002A000113041250E30A100AF2408008030112507
:1002B000A801A7012824403011259C3011250C30BD
:1002C000A70017304C25F8301424F830A4000B3068
:1002D000A7001E304C251030A10024081424051E50
:1002E000C42973252D08A702031CA803A10B6D299F
:1002F000051EC4292D08013EA7070318A80A0830C7
:10030000A100210324041424051EC4297325A10B74
:100310008129A70A0830A100210324041424051E02
:10032000C4297325A10B8C29051EC4291030A100F6
:1003300024081424051EC42973252D08A7070318B3
:10034000A80AA10B9829051EC4292D08A702031C81
:10035000A803A101210824041424051EC42973251F
:10036000A10AA11DAA29A703A1012108240414247C
:10037000051EC4297325A10AA11DB529083024072B
:10038000F038A400051A672908000230A8000030E0
:100390004A251030A100F530A900BC240230A80085
:1003A000063038250930A1000D30A900BC240230E8
:1003B000A800063035250930A1000D30A900BC2465
:1003C000843011259C3011250800973011250F30FD
:1003D000A7000330A800532457240800A8010130C7
:1003E000A7001030A1002824403011250530A000BE
:1003F000051E122A6A25A00BF829A70AA10BF329CA
:100400001130A1001030A7002824403011250530FC
:10041000A000051E122A6A25A00B092AA703A10B1A
:10042000042AEE29080080301125A8011130A70008
:10043000A1012824403011250530A000051E282ADE
:100440006A25A00B1E2AA10AA701A11C192A152A98
:100450000800803011259C301125A8010030A7002C
:100460002824403011250230A80000304A251030E1
:10047000A100A901BC240230A800063038250930AB
:10048000A100A901BC240230A8000630352509309E
:10049000A100A901BC24A8010030A70028244030F5
:1004A00011250F30A2000130A70022084C250A3088
:1004B000A100AA30221C5530A900BC24A20A22089F
:1004C000213A031D532A813011259C301125080043
:1004D000672479241030AD0045244C248030112548
:1004E0009C301125A8010130A7004A250930A10040
:1004F0001030A000AF24A8010B30A7004A2504301B
:10050000A1001E30A000AF2403178D010313A20128
:10051000A3012308A70014304C252030A0005A2541
:1005200019242D08A7070318A80AA00B8F2AA30ACD
:10053000231E892A0317CA308D0003130330A1003C
:100540001430A8008030A7002F24B03011255A2580
:1005500023248D0AA10BA72AB23011253330A30022
:100560000C30A2000030A70023084C251030A10059
:10057000AA30A900BC24A30AA20BB22A1C30A300F3
:10058000343084008001840AA30BC22A0630AE00F6
:100590000130AC001730A300A70123084C252F24FD
:1005A000343084001030A2001C25800DAB0C800C70
:1005B000B0301125D2242B080225B2301125A20B10
:1005C000D42A051E0800840AA30A2308333A031D0F
:1005D000D22AAC03031DCA2AA8012E083E2590305A
:1005E0001924A8010530A70047250530A1003030A7
:1005F000A000AF240330A0006A25A00BFC2AA801AC
:100600000530A70047250530A1000030A900BC2413
:10061000A8012E08A7003E2500301924AE0A2E128C
:100620000830AC002E080319AC0ACA2A94301125F0
:10063000A801A7012F24B0301125A00120082324F0
:10064000A00AA01F1E2BB2301125080003178D0130
:1006500003131430A8008830A7002F24B0301125D0
:10066000A001E030A10020085A252324A00AA10BF4
:10067000332BB2301125A801A7012F24B03011254A
:100680008030A00020082324A00F422BB230112577
:10069000080067249C301125A8010130A7004A25D5
:1006A0000930A1001030A000AF24A8010B30A70032
:1006B0004A250430A1001E30A000AF241030A20053
:1006C000343084008001840AA20B622BAC01AF019C
:1006D000A301A801A7012C08B0002F02031C742B52
:1006E0002F08B0002C08AF002F08E620B1002F0D16
:1006F000B200320E0F39B2003208343E84000310CB
:100700002F08A20022082F060319932B310880041A
:10071000A20AA21BA42B0310B10C031C822B840A77
:10072000B1170310822B220830060319A42B3108BD
:100730008004A20AA21BA42B0310B10C031C932B50
:10074000840AB1170310932B34308400A201A7014F
:1007500023084C252F24B0301125000802258001E4
:10076000840AA20A221EAD2B2C08AF00B23011253C
:100770000430AC07AC13051E0800A30A2308403A56
:10078000031D692BAC03682B9C301125AC01AF0114
:10079000A2018030B1002C08B0002F02031CD42B22
:1007A0002F08B0002C08AF0034302F0784002F082A
:1007B000A30031088004230830060319E62B310812
:1007C0008004A30A231BE62B840ADB2B2C08AF0032
:1007D0000230AC072C130310B10C031CCB2B3430AC
:1007E00084004030A3000230A8002208A7002F2474
:1007F000B0301125D224000802258001B230112525
:10080000840AA3030319092C2D08A7070318A80AB3
:10081000F72BA20A221EC92BA20103302C023F395A
:10082000AC00051AC92B0800AA002F242A0811259C
:100830000800A9002F24B0301125D2242908022550
:10084000B23011250800A500F32425080225080070
:10085000D22427080225D224280802250800D22401
:1008600027080225D2242808022524301125080053
:10087000A801A70128244030112508000230A80053
:10088000A7012824423011250800A8012D08A7003F
:100890002824413011250800A8012D08A70028248C
:1008A0004330112508002824213011250800A730E5
:1008B00011250800803011250800A8010230A7008A
:1008C0002824223011250800943011250800A801A1
:1008D000A7012F24B03011250830A1002D08A00059
:1008E00000302324A00B702CA10B6E2CB2301125EC
:1008F00008000230A800A7012F24B0301125403095
:10090000A1002D08A00000302324A00B832CA10BF4
:10091000812CB230112508001430A800A7012F2423
:10092000B03011254030A1002D08A0000030232454
:10093000A00B962CA10B942CB2301125080014307A
:10094000A800A7012F24B0301125A00120086D2098
:100950002324A00AA10BA62CB230112508002F24B5
:10096000B030112520081C20E03E2324A00AA10B52
:10097000B22CB230112508002F24B03011252908DF
:100980002324A10BBF2CB230112508002F24B03036
:100990001125200852202324A00AA10BC92CB23013
:1009A000112508008316FF30880083121930870054
:1009B0000000081CD92C881CDB2C1F30870000008D
:1009C00083168801831208008316081783121930D2
:1009D00087000000081BEA2C1F30870000008316E8
:1009E00008138312080083168815831219308700B4
:1009F0000000881DF92C1F30870000008316881125
:100A000083120800A5001730870025088800000021
:100A10001230870000001730870000001F30870069
:100A20000800A500D2242508880000001A3087009D
:100A300000001F3087000800E03011258316FF30CA
:100A400088008312193087000000081B252D081C20
:100A5000272D881C292D871100000808AB001F30A6
:100A6000870083168801831208002D070318A80A3F
:100A70002D070318A80A2D070318A80A2D07031825
:100A8000A80A2D070318A80A2D070318A80A2D077E
:100A90000318A80AA7000800A0000230A800200838
:100AA000031908002D08A70701300305A807A00BAC
:100AB000522D0800031783168C130C1483120C0894
:100AC0008D0A03130800051A632D6A25051E662D7D
:100AD0006A2508000530A6008B010B1D6D2D0B113A
:100AE000A60B6D2D08000130A6008B010B1D6D2D8E
:100AF0000B11A60B762D08001F30870038243E24EA
:100B000045244C245A245D246424672479248C24AD
:020B10000800DB
:00000001FF
